:03000000022C537C
:0C2C530078FFE4F6D8FD75816E022C9A23
:100EE20020000A3C2E2E2E3E004950436F6E6E6546
:100EF20063745245510A004950436F6E6E656374C4
:100F0200000A49504E6F41434B210A003E432C5682
:100F12002C43432CC0E4E0EFF2E5F020D1E8EDEA07
:100F2200EEEC49500A003E432C4D41432C25303211
:100F320062583A25303262583A25303262583A25A0
:100F4200303262583A25303262583A25303262588D
:100F52002C4D414320E0E4F0E5F10A003E432C56DB
:100F620045522C20332E3220EEF220257320257399
:100F72002CC2E5F0F1E8FF20495020ECEEE4F3EB5F
:100F8200FF0A004D61722031382032303130003199
:100F9200353A33343A3533003E432C4C442C5052CC
:100FA2004F473A20202020202020202020202020CF
:100FB200202020202020202020202020202020202F
:100FC200202020202020202020202020202020201F
:100FD200202020202020202020202020202020200F
:100FE20020202020202020202CC4E0F2E020EFF05E
:100FF200EEF8E8E2EAE828F4E0E9EB290A003E2A02
:101002002C312CCEF1EDEEE2EDFBE520EFE0F0E04D
:10101200ECE5F2F0FB20F1E5F2E5E2EEE3EE20E8AA
:10102200EDF2E5F0F4E5E9F1E00A003E412C413051
:10103200312C2562752E2562752E2562752E25624C
:10104200752C495020E0E4F0E5F120E0E4E0EFF215
:10105200E5F0E00A003E412C4130322C2562752E2B
:101062002562752E2562752E2562752C495020E069
:10107200E4F0E5F120EEF1ED2E20F1E5F0E2E5F00D
:10108200E00A003E412C4130332C2562752E256248
:10109200752E2562752E2562752C495020E0E4F0EC
:1010A200E5F120F0E5E72E20F1E5F0E2E5F0E00AD7
:1010B200003E412C4130342C2562752E2562752E5E
:1010C2002562752E2562752CCCE0F1EAE020F1E56F
:1010D200F2E80A003E412C4130352C2562752E255E
:1010E20062752E2562752E2562752CD8EBFEE70AF5
:1010F200003E2A2C312CC4EEEF2E20EFE0F0E0EC83
:10110200E5F2F0FB20F1E5F2E5E2EEE3EE20E8EDB8
:10111200F2E5F0F4E5E9F1E00A003E422C53303109
:101122002C2562752CC6E4E0F2FC20E7E0EFF0EE3D
:10113200F1E020F1EEE5E4E8EDE5EDE8FF20EEF286
:1011420020F1E5F0E2E5F0E00A003E422C533032B5
:101152002C2562752CCEE1ECE5ED20F120F1E5F0D5
:10116200E2E5F0EEEC20E1E5E720EAE2E8F2E0ED8C
:10117200F6E8E90A003E422C5330332C2562752CE6
:10118200CFE5F0E5E7E0EFF3F1EA20EFF0E820EF5A
:10119200EEF2E5F0E520F1E2FFE7E820F120F1E5EB
:1011A200F0E2E5F0EEEC0A003E454E440A000A4445
:1011B200756D7058202020202030302030312030B2
:1011C2003220303320303420303520303620303752
:1011D2002030382030392030412030422030432026
:1011E2003044203045203046000A3A003A20000AB6
:1011F200000A44756D7044202020202030302030B9
:101202003120303220303320303420303520303617
:1012120020303720303820303920304120304220F1
:101222003043203044203045203046004572722041
:101232006B657900526420656570726F6D0A0052A9
:1012420064204D454D0A00526420436F64650A00D4
:10125200577269746520436F64650A00446562755C
:10126200674950204F4E0A00446562756749502015
:101272004F46460A00446562756755736572204F92
:101282006E0A00446562756755736572204F464663
:101292000A0044656275674D7367204F6E0A004409
:1012A200656275674D7367204F46460A00436F6E4D
:1012B200666967206C6F636B210A0057722065654F
:1012C20070726F6D0A0020536176652065657072D9
:1012D2006F6D210A00457272204D414321004C6F0F
:1012E20061643E3E002A003C4130313D003C4130C9
:1012F200323D003C4130333D003C4130343D003C06
:101302004130353D003C21003C5330313D003C53DF
:1013120030323D003C5330333D003C5330353D00CC
:061322003C5330363D0093
:06348300016B000169006D
:10350000C28E438910E4F58B758DB8D2ABD28E2272
:03001B00022BC3F2
:102BC300C0E0C083C082C0D0C28E758B00758DB843
:102BD30020060675A61E75A6E10569D202E56B609F
:102BE30002056BE56AD394014002156A056EE56E32
:102BF300540F7048D20EE56E543F7012D2009066A7
:102C03008BE0600A04F0E0D394B44002D2069066ED
:102C130086E0600204F0906104E0600214F09066C4
:102C23008CE0D394014003E014F0300502056CE519
:102C33006DD394644004D2068002056DE568D39495
:102C43000140021568D28ED0D0D082D083D0E0323A
:10087900C291C290D2B5C20B7D027C007F071234AF
:10088900668F25E525646060097D017F601234016A
:10089900D20BE4FDFC7F0B1234668F25E52530E68B
:1008A900097D04E4FF123425D20B7D017C007F070A
:1008B9001234668F25E5257008FD7FFF123401D2B9
:1008C9000B300B03126000C288C2A8C2AA75890046
:1008D900122F7B90633EE0B4FA06A3E064CE607BFE
:1008E900E4F52574362525F582E43463F583E4F0CF
:1008F9000525E525B443EC90633E74FAF0A374CE64
:10090900F0A374CCF0906344740AF0E4A3F0A30458
:10091900F0A3F090633A74FFF0A3F0A3F0E4A3F01E
:10092900906355740AF0E4F525E5252401FFE433C5
:10093900FE74362525F582E43463F583E0FD123330
:10094900DD0525E525C3944340DFE4F5A775A61E1B
:1009590075A6E1907FF0F0A3F080FE9063497403DF
:10096900F0A374CCF0E4906348F01228FDC2B512EC
:1009790034B9C2061231F8D20BC20DC20C90657699
:100989007408F09062B47424F0E4A3F090633EE03C
:100999009062B6F090633FE09062B7F0906340E0F8
:1009A9009062B8F0906341E09062B9F0906342E0E0
:1009B9009062BAF0906343E09062BBF0756A01E41B
:1009C900906577F0C207C208C209C20A200B18AFA6
:1009D90025FE7D03122741E4FF122A7C7E0E7FE269
:1009E900E4FBFDFC12226490668BE060037401F065
:1009F900E4906104F0F56C906575F0F56D123500C1
:100A090075A70775A61E75A6E1D2AFE4F56D9061CD
:100A190004E07003121E0990668CE06401701D9059
:100A290080007410F09080A874FFF0A3F0A3F0A3E5
:100A3900F0E490668CF0D20BC20CC20D908008E0F5
:100A4900F52530E405D2077410F0E52530E508D224
:100A5900099080087420F0E52530E608D2089080D6
:100A6900087440F0E56CC394034019908002E4F0E7
:100A7900908001F0908000F0E56C94064006E4F562
:100A89006C1231F89080A0E070031230739080B836
:100A9900E07003122FF99080D0E0700312319C901E
:100AA9008000E0701330071012236B906331EFF070
:100AB900D394004003120036908002E070069080C3
:100AC90000E06005D205020A14C205E4F56C9061E4
:100AD90004E06003020A14200B12906578E0600CB0
:100AE9007E0E7FE4122659E4906578F030091212DF
:100AF9001F8C906331EFF0D394004005E0FF12356D
:100B090026200803020C8A121C82906331EFF070D0
:100B190003020A14906375E054BF247F7003020B2B
:100B2900F3147003020BCB24026003020C2C200B7C
:100B3900077E0E7FEB122659200F03020C8A906361
:100B49004DE07006906351E06067906682E0FF9027
:100B5900634DE0B50724906683E0FE90634EE0B5EF
:100B69000618906684E0FE90634FE0B5060C906627
:100B790085E0FE906350E06E6037906351E06F60EE
:100B890003020C8A906683E0FF906352E06F600372
:100B9900020C8A906684E0FF906353E06F60030261
:100BA9000C8A906685E0FF906354E06F6003020C45
:100BB9008AC2039065777401F012352C756A0102B7
:100BC9000C8A90668BE060037401F090667AE0FF0E
:100BD900906377E06F6003020C8A90667AE004F014
:100BE900E4F56A906575F0020C8A300303020C8AF9
:100BF900906344E07003020A14906355740AF0127A
:100C090034D3D203E4F56A906575F090668604F0F2
:100C1900E4906679F0A3F0200B677E0E7FF9122627
:100C290059805E90668BE060037401F03003529046
:100C39006375E020E74B906377E0FF906679E0FE0B
:100C49006F600D906681E07007EE146F703380134A
:100C5900906679E004F0906331E0FFD39404400397
:100C69001235299060007482F0A37401F0906377C3
:100C7900E0906002F07E607F007D03122D66020A1B
:100C890014200303020DA2E56A7068123252EF6064
:100C9900237E647F75906476E02404FD122D6690AE
:100CA9006681E07009906355E0F56A020A14E4F57B
:100CB9006A020A14906686E0D3943C4036906681B5
:100CC900E0703090668604F01229C7E4906475F0EC
:100CD900A37412F090667AE0906477F0A374FDF043
:100CE90090610563A20190647963A2017F121219D0
:100CF900D0809E12351B8F25E525B4011590600023
:100D09007483F0E4A3F07E607F007D02122D6602F9
:100D19000A14E525D39401401C9060007483F0A364
:100D29007401F0E52524FEA3F07E607F007D0312A7
:100D39002D66020A14E56A64016003020A149065CB
:100D490075E004F0200B077E0F7F0312265990638C
:100D590055E0C394C85004E02432F0906575E0C3AF
:100D69009405400DC203E4906577F012352C020A10
:100D7900147C667D82906349E0FAA3E0FB7F02124E
:100D89002EF77E647F75906476E02404FD122D664B
:100D9900906355E0F56A020A14E56A64016003028A
:100DA9000A14906577E014604624FE6042147003CB
:100DB900020E9524046003020A14E4F56C200F1353
:100DC9009065777404F0906575E05401F0756A01D7
:100DD900020A149080027410F0E4906577F090652F
:100DE9007504F0756AFA90668274FFF0020A14902D
:100DF9006682E07003020E7F9064757480F09064DF
:100E0900777401F0E4A3F0A304F0A37430F0A374A1
:100E19007BF0E4F525747C2525F582E43464F583BB
:100E2900747DF0747D2525F582E43464F583E4F05E
:100E3900E5252407906476F07C667D82906349E01D
:100E4900FAA3E0FB7F02122EF77E647F75E5252465
:100E590009FD122D66906681E0601B1234D3D2031E
:100E6900E4F56A906575F090668604F0E490667919
:100E7900F0A3F0020A14300F07E4906577F08006BA
:100E89009065777404F0756AFA020A149080027406
:100E990010F0756A05906575E06401FFF09065775B
:100EA9007401F0EF7019906351E06013FCA3E0FD49
:100EB900A3E0FEA3E0FF906682121771020A149064
:100EC900634DE0FCA3E0FDA3E0FEA3E0FF90668292
:080ED900121771020A1480FED9
:010EE10022EE
:10003600906376E0B444047F0180027F009063758C
:10004600E0B447047E0180027E00EE5F604A906362
:100056003EE0906377F090633FE0906378F09063C2
:1000660040E0906379F0906341E090637AF09063AA
:1000760042E090637BF0906343E090637CF0906392
:10008600767452F09062AE63A2019080A863A201DA
:100096007F061219D002086F906331E0C3940850AE
:1000A6000302087890633EE0FF906377E06F600399
:1000B60002087890633FE0FF906378E06F60030288
:1000C6000878906340E0FF906379E06F6003020870
:1000D60078906341E0FF90637AE06F6003020878EE
:1000E600906342E0FF90637BE06F600302087890C4
:1000F6006343E0FF90637CE06F60030208789063DF
:1001060076E06444701A9080A8E0B4FF139062AE63
:1001160063A2019080A863A2017F061219D0801005
:100126009062B2E09080ACF09062B3E09080ADF067
:1001360090668BE060037401F090668C7464F090B6
:1001460063767452F0906375E0646D600302027921
:100156007BFF7A0F790E12138A7BFF7A0F7928902C
:10016600633EE0F532A3E0F533A3E0F534A3E0F512
:1001760035A3E0F536A3E0F53712138A7532FF751D
:10018600330F7534857535FF75360F7537917BFFDF
:100196007A0F795E12138A7BFF7A0F799A12138A85
:1001A6007BFF7A10790012138A7BFF7A10792D90E3
:1001B6006344E0F532A3E0F533A3E0F534A3E0F5BC
:1001C6003512138A7BFF7A10795790634DE0F5322A
:1001D600A3E0F533A3E0F534A3E0F53512138A7BEB
:1001E600FF7A107985906351E0F532A3E0F533A3E9
:1001F600E0F534A3E0F53512138A7BFF7A1079B364
:1002060090633AE0F532A3E0F533A3E0F534A3E0DA
:10021600F53512138A7BFF7A1079D6906336E0F5AE
:1002260032A3E0F533A3E0F534A3E0F53512138AE3
:100236007BFF7A1079F312138A7BFF7A11791CA25D
:100246000FE433F53212138A7BFF7A11794C9066EC
:1002560081E0F53212138A7BFF7A11797790668BEB
:10026600E0F53212138A122B2C7BFF7A1179AA122F
:10027600138A22906375E0644C70737E117FB0FB25
:10028600FDFC12226490637DE0F526A3E0F527E4E9
:10029600F529E52690637FF0A3E527F07E117FEB35
:1002A6007C637D7F7B02122264E4F52885278285A4
:1002B6002683E0FF747F2528F582E43463F583EF17
:1002C600F00527E527700205260528E528B410DC89
:1002D6007E117FEE7C637D7F7B101222640529E50B
:1002E60029C3941040AC7E117FF1122659229063E7
:1002F60075E0646C7060F52A7E117FF3FBFDFC12DD
:100306002264E4F529E490637FF0A3E52AF07E11E8
:100316007FEB7C637D7F7B02122264E4F528A82AAA
:10032600E6FF747F2528F582E43463F583EFF00554
:100336002A0528E528B410E67E117FEE7C637D7FD2
:100346007B101222640529E529C3940840B77E1163
:100356007FF112265922906375E0644B7061F5288F
:1003660074672528F582E43463F583E060327467A8
:100376002528F582E43463F583E0F4602374672569
:1003860028F582E43463F583E0FF747D2528F58241
:10039600E43463F583E0B507100528E528B408C002
:1003A6009061047432F002086F9063757421F03026
:1003B6000B0302086F7E127F2E12265902086F90D9
:1003C6006375E0B4521A200B077E127F3612265947
:1003D6009063757472F07E637F757D08122CDF2240
:1003E600906375E064497045200B077E127F4112C9
:1003F600265990637DE0F526A3E0F527E4F52885E8
:100406002782852683E0FF747F2528F582E43463FE
:10041600F583EFF00527E527700205260528E52870
:10042600B480DC7E637F757D8A122CDF2290637533
:10043600E064437046200B077E127F4912265990CE
:10044600637DE0F526A3E0F527E4F5288527828578
:100456002683E493FF747F2528F582E43463F583CD
:10046600EFF00527E527700205260528E528B48064
:10047600DB7E637F757D8A122CDF22906375E064D4
:100486005A7053200B077E127F5212265990637DB5
:10049600E0F526A3E0F5277C637D7F7B80AF27AE62
:1004A600261233A9E4F528852782852683E493FF5F
:1004B600747F2528F582E43463F583EFF00527E59C
:1004C60027700205260528E528B480DB7E637F7544
:1004D6007D8A122CDF22906375E064446003020576
:1004E6006D90637DE0FF6444700302086FEFB431E2
:1004F6000CC20B7E127F5E12265902086F90637D36
:10050600E0B4300CD20B7E127F6A12265902086FB5
:1005160090637DE0B4320CD20C7E127F771226599E
:1005260002086F90637DE0B4330CC20C7E127F85A7
:1005360012265902086F90637DE0B4340CD20D7E0A
:10054600127F9412265902086F90637DE0B4350C31
:10055600C20D7E127FA112265902086F90637DE0BC
:10056600FF12001E02086F906104E07013200B0753
:100576007E127FAF1226599063757421F002086FC0
:100586009061047432F0906375E0FFB45104C2AF19
:1005960080FEEF64577045200B077E127FBD122642
:1005A6005990637EE0906331F0E4F528906331E082
:1005B600FFE528C39F400302086F747F2528F58254
:1005C600E43463F583E0FF90637DE0252824ADF5F0
:1005D60082E43461F583EFF0052880D0906375E0FE
:1005E60064536003020690200B077E127FC8122612
:1005F6005990633EE0FF9061B6E06F703C90633FB8
:10060600E0FF9061B7E06F7030906340E0FF90616B
:10061600B8E0B50724906341E0FF9061B9E0B50703
:1006260018906342E0FF9061BAE0B5070C9063430F
:10063600E0FF9061BBE06F60169063757421F03047
:100646000B0302086F7E127FD712265902086FE449
:10065600F528E4F56DAF28FE74AD2528F582E4345F
:1006660061F583E0FD1233DD0528E528C394FE40DD
:10067600E1C2AFE4907FF0F0A3F0907FFD74AAF0A2
:10068600A374FFF0A37455F080FE906375E0644F89
:10069600704C90637DE0F526A3E0F527E527452617
:1006A600700A200B077E127FE0122659200B077E68
:1006B600127FE7122659E4F528747F2528F582E48F
:1006C6003463F583E0852782852683F00527E527B1
:1006D600700205260528E528B480DE02086F9063BF
:1006E60075E0FFB4452190637DE0FDA3E0907FF0C7
:1006F600CDF0A3EDF0C2AF907FFD74AAF0A374FF16
:10070600F0A37455F080FEEF6465600302087890EC
:10071600637DE0FFA3E0907FF0CFF0A3EFF0E4F578
:1007260026F527D3907FF1E09527907FF0E0952678
:100736004020E4F56D2527FFE5263401FE85278256
:10074600852683E0FD1233DD0527E52770020526A1
:1007560080D17E127FE9122DEDEF4E60201200034C
:10076600906344EFF0120003906345EFF01200032C
:10077600906346EFF0120003906347EFF07E127F1E
:10078600EF122DEDEF4E602012000390634DEFF057
:1007960012000390634EEFF012000390634FEFF0E8
:1007A600120003906350EFF07E127FF5122DEDEFED
:1007B6004E6020120003906351EFF0120003906325
:1007C60052EFF0120003906353EFF01200039063B0
:1007D60054EFF07E127FFB122DEDEF4E60201200DB
:1007E6000390633AEFF012000390633BEFF01200C0
:1007F6000390633CEFF012000390633DEFF07E132D
:100806007F01122DEDEF4E6020120003906336EF4C
:10081600F0120003906337EFF0120003906338EF95
:10082600F0120003906339EFF0E4F528E4F56DE586
:10083600282401FFE433FE74362528F582E4346368
:10084600F583E0FD1233DD0528E528C3944340DC3B
:10085600C2AFE4907FF0F0A3F0907FFD74AAF0A3FE
:1008660074FFF0A37455F080FE7E637F757D0812D9
:020876002CDF75
:01087800225D
:10337100AE07EEC39430400BEED394395005EE24E2
:10338100D0FF22EEC39461400BEED394665005EE5C
:1033910024A9FF22EEC39441400BEED3944650057D
:0833A100EE24C9FF22AF062251
:10349F009062ADE004F070069062ACE004F09062D0
:0A34AF00ACE0FEA3E0FF1234492256
:1000030012349F123371EFC454F0FEC00612349FB2
:08001300123371D0E02FFF222F
:10313F00E490683AF012349F90683BEFF0C39430FC
:10314F004018E0FFD39439501190683AE02405F508
:10315F0082E43461F583EFF0801190683AE0240542
:10316F00F582E43461F583E4F0800C90683AE00472
:10317F00F0E0D3940840BE752900752A00752B0026
:0C318F00E4F52C7B017A617905121ADE50
:01319B002211
:042DED008E2B8F2C6E
:102DF1009062ACE4F0A374FFF012349FEF606EF4C4
:102E0100606B852C82852B83E493B507EC752D01CE
:102E1100E52C252DF582E4352BF583E4936025908F
:102E210062ADE0252DFF9062ACE03400FE12344922
:102E3100E52C252DF582E4352BF583E493B50704C4
:102E4100052D80CCE52C252DF582E4352BF583E489
:102E51009370A6E52D24FFFFE434FFFE9062ADE000
:102E61002FF09062ACE03EF07E007F0122E4FEFF95
:012E7100223E
:1028FD007E137F07122DEDEF4E70037F01227E13A5
:10290D007F0A122DEDEF4E600C12349FEF24D02470
:10291D00FF920F8002D20F7E137F10122DEDEF4E1E
:10292D00600C12349FEF24D0906681F08005E49006
:10293D006681F07E137F16122DEDEF4E600C123472
:10294D009FEF24D090668BF08005E490668BF07E2F
:10295D00137F1C122DEDEF4E600C12349FEF24D01F
:10296D0024FF92018002C20190633E63A201906632
:10297D007B63A2017F061219D030013B7E137F22AB
:10298D00122DEDEF4E603012000390667BEFF012CA
:10299D00000390667CEFF012000390667DEFF0125D
:1029AD00000390667EEFF012000390667FEFF01249
:0A29BD000003906680EFF07F002217
:1032AB00906576E0C3947C40027F0A906576E0FEE1
:1032BB0004F074B42EF582E43462F583EFF0BF0AA8
:1032CB0027906576E0FF04F074B42FF582E4346246
:1032DB00F583E4F0906576E0FF122E7290657674BC
:0932EB0008F09062B5E004F02245
:1031F8009080007480F090633663A201F583F582B5
:1032080063A2017F081219D090633E63A2019080E7
:103218008863A2017F0A1219D09080927407F0A3E4
:1032280074D0F0A37406F0906348E0FF9080B1F08A
:103238009080E1EFF09080957455F0A3F0908000B5
:0A3248007401F090800974F0F02288
:10307300908009E04410F09080A0E070609080A1FF
:103083007482F09080A874FFF0A3F0A3F0A3F07F04
:10309300039080AEEFF0A374CBF09080007402F045
:1030A30090682A12177D0000000090682AE0908043
:1030B30040F090682BE0908041F090682CE0908085
:1030C30042F090682DE0908043F0A3E4F0A3F0A3D6
:0D30D300F0A3F0908018F0A3F0A3F0A3F09C
:0130E00022CD
:10319C00908009E04440F09080D17482F07F0390DD
:1031AC0080DEEFF0A374CCF09080027402F0906893
:1031BC002E12177D0000000090682EE0908058F0D1
:1031CC0090682FE0908059F0906830E090805AF031
:1031DC00906831E090805BF0A3E4F0A3F0A3F0A33F
:0B31EC00F0908030F0A3F0A3F0A3F0FF
:0131F70022B5
:102FF900908009E04420F09080B8E0706C9080B92E
:103009007482F07F039080C6EFF07FCDA3EFF07F4D
:10301900039080C4EFF0A374CDF09080C074FFF0EA
:10302900A3F0A3F0A3F09080017402F0906832122B
:10303900177D00000000906832E090804CF09068A5
:1030490033E090804DF0906834E090804EF09068C5
:1030590035E090804FF0A3E4F0A3F0A3F0A3F09043
:093069008024F0A3F0A3F0A3F011
:01307200223B
:102EF7008C268D27A907EAFDE975F018A424ACFFF5
:102F0700E5F034808F82F583EDF0EBFDE975F0187D
:102F1700A4FFAEF024ACFBEE34808B82F583A3EDE7
:102F2700F08527828C83E0FDEF24A8FFEE3480FE36
:102F37008F82F583EDF08527828C83A3E08F828EC5
:102F470083A3F0852782852683A3A3E0FDE975F097
:102F570018A424A8FFE5F03480FE8F82F583A3A38D
:102F6700EDF08527828C83A3A3A3E08F828E83A3B2
:042F7700A3A3F022FE
:062CDF008D2BAB07AA06D5
:102CE500908000E030E5079065787401F0229068E7
:102CF5002AE0FCA3E0FDA3E0FEA3E0F52F8E2E8DD8
:102D05002D8C2CAE02AF038E838F8263A201E52E3C
:102D1500540744C0F583852F8263A201AF2B121A95
:102D250042E4FCFDFEE52F252BF52FEE352EF52E85
:102D3500ED352DF52DEC352CF52C908040E52CF05E
:102D4500A3E52DF0A3E52EF0A3E52FF09080007408
:102D550020F0AF2FAE2EAD2DAC2C90682A12177136
:012D6500224B
:062D66008D26AB07AA0652
:102D6C00908002E030E5079065787403F02290685B
:102D7C002EE0FCA3E0FDA3E0FEA3E0F52A8E298D56
:102D8C00288C27AE02AF038E838F8263A201E529C4
:102D9C00540744D0F583852A8263A201AF26121A08
:102DAC0042E4FCFDFEE52A2526F52AEE3529F52917
:102DBC00ED3528F528EC3527F527908058E527F0D8
:102DCC00A3E528F0A3E529F0A3E52AF0908002748E
:102DDC0020F0AF2AAE29AD28AC2790682E121771BF
:012DEC0022C4
:022A7C008F26A3
:102A7E00908001E030E5099065787402F07F0022C5
:102A8E00906832E0FCA3E0FDA3E0FEA3E0F52A8E01
:102A9E00298D288C2790667B63A201E52954074473
:102AAE00C8F583852A8263A2017F06121A58E52A89
:102ABE002406F52AE43529F529E43528F528E435E8
:102ACE0027F52790657963A201E529540744C8F5D7
:102ADE0083852A8263A201AF26121A58E4FCFDFEFA
:102AEE00E52A2526F52AEE3529F529ED3528F5288E
:102AFE00EC3527F52790804CE527F0A3E528F0A3C9
:102B0E00E529F0A3E52AF09080017420F0AF2AAEFB
:0D2B1E0029AD28AC27906832121771AF2640
:012B2B002287
:10236B009081E0E0F526052605260526052605269F
:10237B0005260526052605260526908010E0F5295D
:10238B00A3E0F52AA3E0F52BA3E0F52C9081E1E087
:10239B00F5260526052605260526052605260526EA
:1023AB00052605260526908014E0F52DA3E0F52ED5
:1023BB00A3E0F52FA3E0F530E52FB52B08E530B5FD
:1023CB002C037F0022E4F526E52F540744E0F58328
:1023DB0085308263A20190637563A2017F08121A94
:1023EB008890637763A2019062AE63A2017F0612AD
:1023FB0019D0906375E0F527A3E0F528E4F5269056
:10240B006375E0702AA3E024F8F526E52F54074402
:10241B00E0F58385308274082582F582E43583F5F7
:10242B008363A20190637563A201AF26121A88AE73
:10243B0027E4FCFDE5302528F530E52F3EF52FEDA3
:10244B00352EF52EEC352DF52D908014E52DF0A3C2
:10245B00E52EF0A3E52FF0A3E530F090800074405B
:03246B00F0AF26A9
:01246E00224B
:101C82009081E6E0F5260526052605260526052689
:101C920005260526052605260526908028E0F52935
:101CA200A3E0F52AA3E0F52BA3E0F52C9081E7E071
:101CB200F5260526052605260526052605260526DA
:101CC20005260526052690802CE0F52DA3E0F52EAD
:101CD200A3E0F52FA3E0F530E4F526E52FB52B0AB6
:101CE200E530B52C05C208021DEEE52F540744F07D
:101CF200F58385308263A20190637563A2017F0838
:101D0200121A88906375E0F527A3E0F528E52845C7
:101D12002770099080027410F07F0022906682E0A2
:101D2200FFF46030906377E06F6003021DB5906648
:101D320083E0FF906378E06F7079906684E0FF90B3
:101D42006379E06F706D906685E0FF90637AE06F73
:101D52006031805F906377E0906682F0906378E014
:101D6200906683F0906379E0906684F090637AE005
:101D7200906685F090637BE0FFA3E0906349CFF02B
:101D8200A3EFF0906375E0702AA3E024F8F526E54E
:101D92002F540744F0F58385308274082582F5823A
:101DA200E43583F58363A20190637563A201AF26D4
:101DB200121A88AE27E4FCFDE5302528F530E52F20
:101DC2003EF52FED352EF52EEC352DF52DAF2CAE43
:101DD2002BAD2AAC29AB30AA2FA92EA82DD31217CE
:101DE2006040099080027410F07F002290802CE500
:101DF2002DF0A3E52EF0A3E52FF0A3E530F09080BF
:061E0200027440F0AF265F
:011E080022B7
:101F8C009081E3E0F526052605260526052605267F
:101F9C000526052605260526052690801CE0F52934
:101FAC00A3E0F52AA3E0F52BA3E0F52C9081E4E067
:101FBC00F5260526052605260526052605260526CD
:101FCC00052605260526908020E0F52DA3E0F52EAC
:101FDC00A3E0F52FA3E0F530E4F526E52FB52B0AA9
:101FEC00E530B52C05C2090220E2E52F540744E880
:101FFC00F58385308263A20190600463A2017F0E99
:10200C00121A9E906004E0F527A3E0F52890600C6E
:10201C00E0FFF4604A90667BE0FEEF6E7079A3E01F
:10202C00FF90600DE06F706F90667DE0FF90600E2A
:10203C00E06F706390667EE0FF90600FE06F70570A
:10204C0090667FE0FF906010E06F704B906680E0D0
:10205C00FF906011E06F703FE4906013F080089087
:10206C00601374FFF0D2D9906004E0702AA3E024CE
:10207C00F2F526E52F540744E8F583853082740E7B
:10208C002582F582E43583F58363A20190600463B5
:10209C00A201AF26121A9EAE27E4FCFDE5302528DE
:1020AC00F530E52F3EF52FED352EF52EEC352DF5D3
:1020BC002DAF2CAE2BAD2AAC29AB30AA2FA92EA854
:1020CC002DD31217605006E5284527700990800122
:1020DC007410F07F0022908020E52DF0A3E52EF007
:1020EC00A3E52FF0A3E530F09080017440F0AF260B
:0120FC0022C1
:042659008E2B8F2C09
:10265D00908000E030E5079065787401F022906875
:10266D002AE0FCA3E0FDA3E0FEA3E0F5328E318D60
:10267D00308C2FE532FFE5315407FEE42FF52EEEB9
:10268D0034C0F52D852E82F5837423F0052EE52EAD
:10269D007002052D532DC7F582852D83740AF00523
:1026AD002EE52E7002052D532DC790633E63A201BA
:1026BD00852D83852E8263A2017F06121A42740630
:1026CD00252EF52EE4352DF52D852B83852C826356
:1026DD00A201852D83852E8263A201121A26E4FCA8
:1026ED00FDFE90682AE0F8A3E0F9A3E0FAA3E02F3D
:1026FD00FFEE3AFEED39FDEC38FCEF2408FFE43E29
:10270D00FEE43DFDE43CFC90682A12177190682AA6
:10271D00E0908040F090682BE0908041F090682C24
:10272D00E0908042F090682DE0908043F090800022
:03273D007420F015
:012740002276
:0A2264008E2B8F2C8C2D8D2E8B2FCE
:10226E00908000E030E5079065787401F022906868
:10227E002AE0FCA3E0FDA3E0FEA3E0F5358E348D4D
:10228E00338C32E535FFE5345407FEE42FF531EE9D
:10229E0034C0F530853182F5837423F00531E53194
:1022AE00700205305330C7F582853083740AF0050D
:1022BE0031E531700205305330C790633E63A201A1
:1022CE0085308385318263A2017F06121A4274061D
:1022DE002531F531E43530F530852B83852C82633D
:1022EE00A20185308385318263A201121A268F36B0
:1022FE00EF2531F531E43530F530E52F6017852DBA
:10230E0083852E8263A20185308385318263A2018B
:10231E00AF2F121A42E5362408252FF52FFFE4FCC5
:10232E00FDFEE5352FF535EE3534F534ED3533F567
:10233E0033EC3532F532908040E532F0A3E533F0E0
:10234E00A3E534F0A3E535F09080007420F0AF35AE
:0C235E00AE34AD33AC3290682A12177117
:01236A002250
:062822008E278F288D298E
:10282800908000E030E5079065787401F0229068A8
:102838002AE0FCA3E0FDA3E0FEA3E0F52F8E2E8D99
:102848002D8C2CE52FFFE52E5407FEE42FF52BEEFB
:1028580034C0F52A852B82F5837423F0052BE52BEC
:102868007002052A532AC7F582852A83EBF0052BC7
:10287800E52B7002052A532AC790633E63A201859F
:102888002A83852B8263A2017F06121A42740625C9
:102898002BF52BE4352AF52A85278385288263A220
:1028A80001852A83852B8263A201AF29121A4274FB
:1028B800082529F529FFE4FCFDFEE52F2FF52FEE6D
:1028C800352EF52EED352DF52DEC352CF52C90808B
:1028D80040E52CF0A3E52DF0A3E52EF0A3E52FF0BD
:1028E8009080007420F0AF2FAE2EAD2DAC2C9068E8
:0428F8002A12177118
:0128FC0022B9
:022E72008F438C
:102E7400908000E030E5079065787401F022906856
:102E84002AE0FCA3E0FDA3E0FEA3E0F5478E468D17
:102E9400458C44E547FFE5465407FEE42FFFEE3436
:102EA400C09062B463A201F5838F8263A201AF4331
:102EB400121A42E4FCFDFEE5472543F547EE35468C
:102EC400F546ED3545F545EC3544F544908040E54F
:102ED40044F0A3E545F0A3E546F0A3E547F0908070
:102EE400007420F0AF47AE46AD45AC4490682A125A
:022EF400177154
:012EF60022B9
:062741008E268F27AB0578
:10274700908000E030E5079065787401F02290688A
:102757002AE0FCA3E0FDA3E0FEA3E0F52D8E2C8D7F
:102767002B8C2AE52DFFE52C5407FEE42FF529EEE7
:1027770034C0F528852982F5837423F00529E529D6
:10278700700205285328C7F582852883EBF00529B1
:10279700E5297002052890633E63A2018528838599
:1027A700298263A2017F06121A4274062529F52998
:1027B700E43528F5285328C7E52685298285288307
:1027C700F00529E529700205285328C7F5828528D1
:1027D70083E527F00529E529700205285328C7E571
:1027E7002D240AF52DE4352CF52CE4352BF52BE4B7
:1027F700352AF52A908040E52AF0A3E52BF0A3E5DA
:102807002CF0A3E52DF09080007420F0AF2DAE2CB6
:0A281700AD2BAC2A90682A1217714D
:012821002294
:0A351000E4FEEEC39F50030E80F8A6
:01351A00228E
:10344900A2AF921DC2AF438E2075D2028F828E83A6
:0C345900E0FFE4F5D2538EDFA21D92AF1D
:013465002244
:1033DD00E5D220E0FBA2AF921DC2AF43D2028F8295
:1033ED008E83EDF075D25063D250A21D92AFE5D20F
:0333FD0020E0FBD2
:0134000022A9
:102F7B00E4FDED2401FFE433FE12344974362DF5E4
:102F8B0082E43463F583EFF00DBD3FE6E4FDED2401
:102F9B007FFFE433FE123449742D2DF582E4346146
:102FAB00F583EFF0742D2DF582E43461F583E07039
:102FBB001B742D2DF582E43461F5837420F0742E8F
:102FCB002DF582E43461F583E4F080040DBD80BE01
:102FDB00E49061ACF0FDEDFF7E0012344974AD2D31
:0D2FEB00F582E43461F583EFF00DBDFEE9E1
:012FF80022B6
:0233A9008B2B6C
:1033AB00A2AF921DC2AF85A22C53A2FE8E838F8239
:1033BB0005A28C838D827409121ACCE52B53A2FEC5
:1033CB0043A220121ACE53A2DF852CA2A21D92AFCC
:0133DB00FFF2
:0133DC0022CE
:10346600A2AF921DC2AF8C838D82EF121ACC43A2FB
:0C34760020121ACE53A2DFA21D92AFFF5D
:013482002227
:023401008F2614
:10340300A2AF921DC2AFE4F5838D827406121ACC6B
:10341300E52643A220121ACE53A2DFA21D92AF7F4C
:0134230001A7
:013424002285
:023425008F26F0
:10342700A2AF921DC2AFE4F5838D82740A121ACC43
:10343700E52643A220121ACE53A2DFA21D92AF7F28
:013447000183
:013448002261
:1018F500A907E7FFA805EF93C3966008403B74FC72
:101905002FFF80F00F08EF93C3966008402B74FB00
:101915002FFF80E00F08EF93C3966008401B74FA11
:101925002FFF80D00F08EF93D3966008400B74F912
:101935002FFF80C01F1F1F1F1FEF54FEF80303F763
:10194500E893FC08E893FD08E893FE08E893FF2276
:1019550009E993C39D6008402974FB29F980F109C1
:10196500E993C39E6008401A74FA29F980E209E9EF
:1019750093D39F6008400B74F929F980D31919197D
:101985001919E9C313C313FF22740093F8ECC39824
:101995004024701F740193F8EDC3984019701474B6
:0E19A5000293F8EEC398400E7009740393F895
:1019B300EFC39840037F00227F0122EDF8E6F00891
:1019C300A3DFFA22EDF8E0F608A3DFFA22E0A3632F
:1019D300A201F0A363A201DFF475A2002263A201B6
:1019E300F0A363A20122E0A363A201F0A363A20117
:1019F300E0A363A201F0A363A201E463A201F0A345
:101A030063A201DFE175A20022E0A363A2016DFEE0
:101A1300936CFDEE058393FC158363A201DFEA75E6
:101A2300A200227F00E493A363A201F00F600CA342
:101A3300E583C2E3F58363A20180EA75A20022E095
:101A4300A363A201F0A3E583C2E3F58363A201DFED
:101A5300EE75A20022E0A363A201F0A3E583C2E432
:101A6300D2E3F58363A201DFEC75A20022E0A36356
:101A7300A201F0A3E58344F8C2E5F58363A201DF85
:101A8300EC75A20022E583C2E3F583E0A363A20120
:101A9300F0A363A201DFEE75A20022E583C2E4D2C4
:0A1AA300E3F583E0A363A201F0A3C2
:101AAD0063A201DFEC75A20022E58344F8F583E023
:101ABD00A363A201F0A363A201DFEE75A20022F9D8
:101ACD0022C002C004C00612FFF0D006D004D0021E
:011ADD0022E6
:10001E00BF360BD217E4F549F54AF565F566BF37DD
:04002E0002C21722D1
:1030E100C2A9438902906825E0FFF58C8F8A75D9C2
:1030F1000475DA4875DB3175DC4975DD4975DE31FA
:10310100E4F5E9F5F9F5EBF5FB906823E060167558
:10311100EC1075ED10E4F5FCF5FD756108755F10B7
:10312100756001801375EC8075ED80E4F5FCF5FDAB
:0E313100756180F55F756010E4F5EEF5FE2225
:10333800E4FEAF8CEFFD906824E07003A3E06D60BD
:10334800051230E17E01E5D920E2057E021230E166
:10335800E58920E1051230E17E03D28C75D84075ED
:08336800B740D2AED2AFAF06B0
:01337000223A
:030033000220FDAB
:0B20FD00C0E0C083C082C0D075D008D6
:10210800C2AF30DC56C3E5EC95EEC395615012E5DD
:102118006025ECF5EC30D70405FC801685FCFC80C6
:1021280011C3E5EC9560F5EC30D70415FC80038508
:10213800FCFC301724854A82854983E590F0054ADE
:10214800E54A70020549F582854983E5EEF0054ABE
:10215800E54A7002054953490FC2DC30D9293017C6
:1021680024854A82854983E590F0054AE54A70024C
:102178000549F582854983E5EBF0054AE54A700291
:10218800054953490FC2D930DA53E55F700405FC9D
:102198008010E55F25ECF5EC30D70405FC8003855D
:1021A800FCFC301836E54B5480F548E54BC313F575
:1021B8004B3097042480F54B201603634B80202670
:1021C8001A0562E5625407701253623FE562131301
:1021D80013541F244DF8A64B754B00C2DA30DB713F
:1021E800E55F700405FD8010E55F25EDF5ED30D75E
:1021F8000405FD800385FDFDE563655E6029E55EF8
:1022080054077013E55E131313541F2455F8E6F5AD
:102218004C201503634CFFE54C139296E54CC31311
:10222800F54C055E535E3FB292301723854A82858E
:102238004983E590F0054AE54A70020549F582852B
:102248004983E4F0054AE54A7002054953490FC23B
:03225800DBD2AF27
:09225B00D0D0D082D083D0E03253
:10246F0042415544005245565F544954003E2A2C70
:10247F00312CCFE0F0E0ECE5F2F0FB20F1E8EDF5E8
:10248F00F0EEEDEDEEE3EE20EFEEF0F2E00A003EBF
:10249F004C2C4230312C256C752CD1EAEEF0EEF13C
:1024AF00F2FC20EEE1ECE5EDE02C35302C31303054
:1024BF002C3230302C3330302C3630302C3132300F
:1024CF00302C323430302C343830300A003E422C2D
:1024DF004731302C2562752CC8EDE2E5F0F1E8FFAD
:1024EF0020EDE020EFF0E8B8ECE50A003E2A2C31B1
:1024FF002CC0E4E0EFF2E5F020F1E8EDF5F0EEEDC1
:10250F00EDEEE3EE20EAE0EDE0EBE02E20CFF0EE93
:10251F00F2EEEAEEEB20D3D2CA2D310A003E422C66
:10252F005430312C2562752CD0E5E2E5F0F120D244
:10253F00C8D20A003C21003C4230313D003C4731BB
:10254F00303D003C5430313D00FF246FFF247400B8
:0F255F0008040C020A060E0109050D030B070FF5
:1034890052668D00000000000000000000000000EE
:0534990000000000002E
:1034EC00EF540F90255E93FEC454F0FEEFC4540FBE
:0434FC00932EFF22EA
:033526008F2622CB
:1034B90090682474FFF0A374B8F0E4906823F0C214
:0A34C9001012256ED21A1230E12213
:1034D300D21490669F7401F0E4F519F515D218C261
:0934E3001CC291C2901233382280
:033529008F2622C8
:10325200301C53E4906475F0A37409F090667AE030
:10326200906477F0A37414F0E4A3F09067A263A2D1
:103272000190647A63A2017F081219D0C21C906681
:103282008FE0FCA3E0FDA3E0FEA3E0FFE4FAF9F87F
:10329200EF2401FFEA3EFEE93DFDE83CFC90668F2B
:0932A2001217717F01227F002246
:101E090030172DC3E54A9566FFE5499565FED3EF81
:101E19009440EE940040197B087D40AF66AE651290
:101E29002822E5662440FFE43565540FF5658F6681
:101E3900301A051234D3C21A201403021F8BE51578
:101E49007003021ED1301903021ED1301205E51AA2
:101E590020E00820120DE51A20E00890669FE004B2
:101E6900F0805AA212B39212E516C313F5169066C2
:101E79009FE024FD600D24FE600E240470115316AA
:101E89007F8013431680800E75190FD2918007D277
:101E990011E4F519C291E51960021519E5191460E3
:101EA9000C24FB70129066A0E516F0800A9066A1DA
:101EB900E516F0D219C29190669F7401F0E51AC334
:101EC90013F51A1515021E4730196FC2199066A12C
:101ED900E0FF5480FEEF25E0F054A0FF9066A0E0FB
:101EE90054AA6FF52630D00BEE6004D21C800DD2B7
:101EF900118009EE7004D21C8002D2119067A2747D
:101F090010F0E4A3F0A3F09066A0E0FE540F9067F0
:101F1900A5F0A37450F0E4A3F0A3F0EEC4540FFFAE
:101F29009066A1E054F02F9067A9F030102AE0FFE5
:101F39001234EC9067A9EFF0801EE5625438655DB4
:101F49006016E55D24085438F55D131313541F24F6
:101F59004DF8E6F51A751508301127906697E0FCDB
:101F6900A3E0FDA3E0FEA3E0FFE4FAF9F8EF240102
:101F7900FFEA3EFEE93DFDE83CFC906697121771C9
:021F8900C21183
:011F8B002233
:0B351B00301B05C21B7F01227F002235
:1029C700E4FF0F2405F582E43461F5837414F00FF6
:1029D70074052401F582E43461F583E4F07C667DB7
:1029E70092FEED1DAA0470011CF5828A83E0FBAA02
:1029F700070F74052AF582E43461F583EBF00EBE08
:102A070004E07C667D96E4FEED1DAA0470011CF5CA
:102A1700828A83E0FBAA070F74052AF582E43461F2
:102A2700F583EBF00EBE04E07C667D9AE4FEED1DB7
:102A3700AA0470011CF5828A83E0FBAA070F7405BC
:102A47002AF582E43461F583EBF00EBE04E07C6680
:102A57007D9EE4FEED1DAA0470011CF5828A83E0C9
:102A6700FBAA070F74052AF582E43461F583EBF0BE
:042A77000EBE04E0AB
:012A7B002238
:102B2C00906823E06022A3E0FEA3E0FFC3E49FFFD4
:102B3C00E49EFEAB07FA3395E0F9F87F007EC27D88
:102B4C00017C001232F48021906824E0FEA3E0FFA7
:102B5C00C3E49FFFE49EFEAB07FA3395E0F9F8E47B
:102B6C007F207E1CFDFC1232F48F2E8E2D8D2C8C32
:102B7C002B7BFF7A24797C12138A7BFF7A24799E33
:102B8C00852E35852D34852C33852B3212138A7B7B
:102B9C00FF7A2479DCA216E433F53212138A7BFF18
:102BAC007A2479FB12138A7BFF7A25792CA210E404
:062BBC0033F53212138A0A
:012BC20022F0
:10256E007E257F43122DEDEF4E70037F01227E25D7
:10257E007F46122DEDEF4E700302261512313F905D
:10258E006836121771E4FFFEFDFC906836E0F8A382
:10259E00E0F9A3E0FAA3E0FBC31217606025906890
:1025AE0036E0F8A3E0A3E0A3E0E47F207E1CFDFC70
:1025BE001216C0121752906824EEF0A3EFF0E490BA
:1025CE006823F0E47FB07E04FDFC906836E0F8A34B
:1025DE00E0F9A3E0FAA3E0FBD3121760403890684D
:1025EE00237401F0906836E0F8A3E0A3E0A3E07F47
:1025FE00007EC27D017C001216C012175290682414
:10260E00EEF0A3EFF0800F90682474FFF0A374B87F
:10261E00F0E4906823F07E257F4C122DEDEF4E6096
:10262E000C12349FEF24D024FF92168002C2167E25
:10263E00257F52122DEDEF4E600C12349FEF24D0F9
:0A264E0024FF92108002C2107F00EA
:01265800225F
:03352C00C2AE220A
:102C5F00020879E493A3F8E493A34003F68001F20A
:102C6F0008DFF48029E493A3F85407240CC8C33376
:102C7F00C4540F4420C8834004F456800146F6DF45
:102C8F00E4800B0102040810204080903483E47E1E
:102C9F00019360BCA3FF543F30E509541FFEE4933A
:102CAF00A360010ECF54C025E060A840B8E493A301
:102CBF00FAE493A3F8E493A3C8C582C8CAC583CA2C
:102CCF00F0A3C8C582C8CAC583CADFE9DEE780BEE4
:01349E00002D
:1016840075F008758200EF2FFFEE33FECD33CDCC1D
:1016940033CCC58233C5829BED9AEC99E5829840A0
:1016A4000CF582EE9BFEED9AFDEC99FC0FD5F0D67D
:1016B400E4CEFBE4CDFAE4CCF9A88222B800C1B9A7
:1016C4000059BA002DEC8BF084CFCECDFCE5F0CBE5
:1016D400F97818EF2FFFEE33FEED33FDEC33FCEB1E
:1016E40033FB10D703994004EB99FB0FD8E5E4F9D9
:1016F400FA227818EF2FFFEE33FEED33FDEC33FCC6
:10170400C933C910D7059BE99A4007EC9BFCE99AB9
:10171400F90FD8E0E4C9FAE4CCFB2275F010EF2FFE
:10172400FFEE33FEED33FDCC33CCC833C810D707FE
:101734009BEC9AE899400AED9BFDEC9AFCE899F839
:0E1744000FD5F0DAE4CDFBE4CCFAE4C8F922CC
:1032F400C2D5E830E70FB2D5E4C39BFBE49AFAE405
:1033040099F9E498F8EC30E717B2D512332A12167B
:10331400C0E4C39BFBE49AFAE499F9E498F88003C7
:103324001216C030D50DE4C39FFFE49EFEE49DFD5C
:04333400E49CFC22F7
:0E175200C3E49FFFE49EFEE49DFDE49CFC22A8
:10176000EB9FF5F0EA9E42F0E99D42F0E89C45F0DF
:011770002256
:0C177100ECF0A3EDF0A3EEF0A3EFF022EB
:10177D00A8828583F0D083D0821217941217941209
:10178D001794121794E473E493A3C583C5F0C5832E
:10179D00C8C582C8F0A3C583C5F0C583C8C582C8B6
:0117AD002219
:10132800E53E2432F8E6053E22782F302402783252
:10133800E475F0011218550217AE201DEB7F2ED26E
:101348001D8018EF540F2490D43440D4FF30210B63
:10135800EF24BFB41A0050032461FFE53F60021573
:101368003F0542E5427002054130240D782FE475AF
:10137800F001121855EF0217F40232AB7403D224AD
:101388008003E4C224F53E8B2F8A308931E4F53F8F
:10139800F541F542E53F60077F2012136380F5753C
:1013A80040FFC21EC21DC21FC220C222C223C225C4
:1013B800121331FF700D3024057F00121374AF42F1
:1013C800AE4122B4255FC2D5C221121331FF24D009
:1013D800B40A00501A75F00A783F30D50508B6FFF0
:1013E8000106C6A426F620D5047002D22080D9248E
:1013F800CFB41A00EF5004C2E5D221021574D21EF0
:1014080080C6D21D80C0D21F80BCD2D580BAD2225D
:1014180080B47F20121363201F077401B53F00407A
:10142800F1121328FF12136302139CD225D22380D2
:1014380095121328FB121328FA121328F94A4B7035
:101448000679457A167BFF201F2EE53F602A7E002D
:101458008E827583001217C760060EEE654070F025
:10146800C2D5EBC0E0EAC0E0E9C0E0EE1215BBD09F
:10147800E0F9D0E0FAD0E0FB1217AEFF60AAEBC0AB
:10148800E0EAC0E0E9C0E0121363D0E02401F9D03B
:10149800E03400FAD0E0FBE5400460DCD540D980B8
:1014A800877BFF7A1579B7D21F809C7910800279E3
:1014B80008C223C2258008D2D5790A8004790AC2D5
:1014C800D5E540047002F540E4FAFDFEFF1213284A
:1014D800FC7B08201E13121328FD7B10301D0A12F6
:1014E8001328FE121328FF7B20EC3382D592D550A7
:1014F80013C3E4301D069FFFE49EFEE4201E039DF7
:10150800FDE49CFCE4CBF8C21EEC700CCFCECDCC35
:10151800E824F8F870F38017C3EF33FFEE33FEEDDD
:1015280033FDEC33FCEB33FB994002FB0FD8E9EBBE
:10153800301E05F8D0E0C448B21EC0E00AEC4D4E9B
:101548004F78207B0070C2EAB5400040BCC0E01272
:1015580015BDD0F0D0E0201E04C4C0E0C4B21EC047
:10156800F012134CD0F0D5F0EB02139C1218B414FF
:10157800395314B358140A4C14064214B74F14BF05
:0F1588004414BF49141F4314C55514A94614A990
:101597004514A947166550140E2D14122E14352B19
:1015A700141623143320164E2A13CE480000142D88
:1015B7003F3F3F00790AA2D5202014302209B910F5
:1015C700020404B9080104A2D52023025001042013
:1015D7001F68921FB53F005034C0E07F20302019AC
:1015E7007F30A21F72237222500F121614C21FC21D
:1015F70023C222C2257F30800F302203E9C0E012C8
:101607001363302203D0E0F9D0E0B53FCC30221786
:101617007F30B9100C1213637F583021077F788011
:1016270003B90803121363301F057F2D0213637F6D
:10163700202025F87F2B2023F322921F80CF286EAE
:10164700756C6C2900D21E121328301EF8C21E7842
:101657003F30D50108F60213CE2D504349581213D7
:10166700282403B405004001E49016609312135434
:0D167700743A121354D220753F040214B3CC
:101ADE008B268A278928E4F532F531F530F52FF576
:101AEE002DF52EE52A452B45296012EBC0E0EAC004
:101AFE00E0E9C0E0AB29AA2AA92B121865AB26058E
:101B0E0028E528AA277002052714F91217AEF53317
:101B1E00C394094007E533D3940D40E1E5336420C7
:101B2E0060DBE533B42D05432E038016E533B42B6D
:101B3E0005432E01800C74FF2528F52874FF3527E8
:101B4E00F527E52C60046410703FAB26AA27A92860
:101B5E001217AE64306009E52C702E752C0A8029A0
:101B6E009000011217C7FF64786004EFB458134356
:101B7E002E01752C1074022528F528E43527F5273B
:101B8E008007E52C7003752C08AB260528E528AADE
:101B9E00277002052714F91217AEF533C39461406E
:101BAE000AE533D3947A50035333DF74D02533F5DB
:101BBE0033C3940A400CE5339411406D74F9253308
:101BCE00F533E533D3952C5060432E01853237859E
:101BDE003136853035852F34AF2C7E00E4FCFDABDD
:101BEE0032AA31A930A82F121806C8ECC8C9EDC9FF
:101BFE00CAEECACBEFCBE4FCFDFEEB2533F532EE9D
:101C0E003AF531ED39F530EC38F52FAF32AE31AD66
:101C1E0030FCAB37AA36A935A834D312176050035F
:101C2E00021B97432E04021B97E52E20E003E4804F
:101C3E002DE52A452B4529601EAB26E52824FFF904
:101C4E00E52734FFFAEBC0E0EAC0E0E9C0E0AB29DB
:101C5E00AA2AA92B121865E52E30E20774FFFFFEA3
:101C6E00FDFC22E52EAF32AE31AD30AC2F30E103AC
:041C7E0002175222D5
:1017AE00BB010689828A83E0225002E722BBFE0239
:0917BE00E32289828A83E493226C
:1017C700BB010CE58229F582E5833AF583E02250D7
:1017D70006E92582F8E622BBFE06E92582F8E22221
:0D17E700E58229F582E5833AF583E493223B
:1017F400BB010689828A83F0225002F722BBFE01D4
:02180400F322CD
:10180600E88FF0A4CC8BF0A42CFCE98EF0A42CFC81
:101816008AF0EDA42CFCEA8EF0A4CDA8F08BF0A4FF
:101826002DCC3825F0FDE98FF0A42CCD35F0FCEB5E
:101836008EF0A4FEA9F0EB8FF0A4CFC5F02ECD3923
:0F184600FEE43CFCEAA42DCE35F0FDE43CFC2290
:10185500FAE6FB0808E6F925F0F618E6CA3AF62294
:10186500BB011A89828A83D0F0D0E0F8D0E0F9D0A4
:10187500E0FAD0E0FBE8C0E0C0F00218E35016E95A
:10188500F8D083D082D0E0F9D0E0FAD0E0FBC08276
:10189500C0830218DABBFE16E9F8D083D082D0E007
:0F18A500F9D0E0FAD0E0FBC082C0830218EC2239
:1018B400D083D082F8E4937012740193700DA3A3C3
:1018C40093F8740193F5828883E4737402936860D7
:0618D400EFA3A3A380DFD7
:0918DA00EBF608EAF608E9F62233
:0918E300EBF0A3EAF0A3E9F02206
:0918EC00EBF208EAF208E9F2222D
:00000001FF
